:106E1F004204030000420408000042040A0000C1BB
:056E2F0013C114C112A3
:0A928200C214C213E490050CF022A0
:108F6200E4900403F0A3F0900408F0A3F090040C42
:108F7200F090040AF0A3F090040604F0A3E4F09049
:048F82000405F022D0
:0692BF00129282028F6290
:10910B00E4F5848FC343C30175C04475CF8EC2C3CE
:09911B0043E60290040104F02275
:10501B00E4F58420C7FDC2C21292BFE4900401F0F4
:01502B002262
:0B923500E4F584D2C290040104F02292
:0D921B00AE0712910B900402EEF00292BF1C
:108F1800E4900686F0A3F0301402FF222013FDD25D
:108F28001490050DE4F0A37410F0900510EFF0E430
:048F3800A3F07F0122
:018F3C002212
:108D820030140A90050DE07002A3E070037F002208
:108D920090050EE024FFF090050DE034FFF0900501
:108DA20011E0FE04F074122EF582E43405F583EF2F
:048DB200F07F01222B
:0B924000301407C214D21312916D22EB
:10916D00900686E584F0E4F58420C7FDC2C4D2C51F
:06917D00900686E0F58477
:0191830022C9
:10877D008B2F8A308931900401E07002FF22E5329F
:10878D006005D3941040037F0022128F18EF6043D1
:10879D00E4900685F0900685E0FFC39532501FAB3F
:1087AD002FAA30A9318F82758300124710FF128DC9
:1087BD0082EF7002FF22900685E004F080D7E490EE
:1087CD00050CF0129240E53370032013FD90050C5B
:0387DD00E0FF2298
:0387E0007FFF22F6
:067328008B2C8A2D892E3A
:10732E00E490067AF0D3900404E09400900403E015
:10733E006480948050037F002253E6FD90040AE09F
:10734E00FEA3E0240CF58274043EF583E090067AE9
:10735E00F090040AE475F001124771FEE4B5F00BEB
:10736E00EEB40107E490040AF0A3F0900407E004E1
:10737E00F07006900406E004F0E490067BF09006B0
:10738E007BE0FFC39D505F90067AE0FEEFC39E50F8
:10739E005590040AE0FEA3E0240CF58274043EF539
:1073AE0083E0FFAB2CAA2DA92E90067BE0F582750B
:1073BE008300EF12474F90040AE475F001124771F3
:1073CE00FEE4B5F00BEEB40107E490040AF0A3F06E
:1073DE00900407E004F07006900406E004F09006B6
:1073EE007BE004F0809890067AE0FFA3E0C39F5004
:1073FE003090040AE475F001124771FAE4B5F00B0F
:10740E00EAB40107E490040AF0A3F0900407E00444
:10741E00F07006900406E004F090067BE004F08025
:10742E00C5900404E024FFF0900403E034FFF04321
:10743E00E602EFC39D500790067AE0FF8002AF058B
:01744E00221B
:10913D00D3900404E09400900403E0648094804094
:08914D00047F0180027F002273
:03501800026CBF68
:106CBF00C0E0C0F0C083C082C0D075D000C000C09B
:036CCF0006C007F5
:106CD200C20AAFC1EF1249B16D08086D08106D18F4
:106CE200186D1D206D2A286D57306D62386D6A60EF
:106CF2006D65686D6A706D65786D72806D72906D8C
:106D0200EBA000006DF9900510E0F5C2C2C5900538
:106D12000FE4F0026DFB900511802890050C74FDC4
:106D2200F0D2C4D2C5026DFB900511E0FF90050FB1
:106D3200E0C39F5014E0FF04F074122FF582E43494
:106D420005F583E0F5C2026DFBD2C490050CE4F0B8
:106D5200C213026DFBD2C590050C74FEF0026DFBEE
:106D6200026DF0D212026DFB900400E4F0026DFBA2
:106D7200900400E07020E5C2F0E0FFC3900407E059
:106D82009F7480F8900406E06480985003128F622A
:106D9200900400E004F0900407E024FFF090040661
:106DA200E034FFF0900408E0FEA3E0240CF58274C6
:106DB200043EF583E5C2F0900408E475F001124741
:106DC20071FEE4B5F00BEEB40107900408E4F0A301
:106DD200F0900400E014F07020900404E004F070DD
:106DE20018900403E004F0801030120DC2129005D6
:106DF2000FE4F0D2C58002D20A300A0EC2C6D2C651
:0C6E0200C2C5C2C4D2C2C20AC213C2C3BD
:106E0E00D007D006D000D0D0D082D083D0F0D0E042
:016E1E003241
:0592C500A2C7E433FF25
:0192CA002281
:088BF9008B298A2A892B8D2C9F
:108C0100E4900683F0AB29AA2AA92B852C32852D65
:108C110033E4FF12877D900684EFF0BFFF0D9006CD
:108C210083E0FF04F0EFC3940340DA900684E0FF91
:028C31007E00C3
:018C3300221E
:068EF2008B298A2A892B5E
:108EF8007E007F007D101249D7AB29AA2AA92B7DB5
:0F8F080010127328900679EFF07002FF227F019C
:018F17002237
:108843009006797422F0A3EFF0A37413F01246F7A5
:1088530090067CF090000112471090067DF0900086
:108863000212471090067EF0900003124710900604
:108873007FF0900004124710900680F090000512DC
:108883004710900681F0900006124710900682F080
:0E8893007B017A067979E4F52D7D0A028BF9D6
:108FEA009006797422F0A3EFF0A37403F0A374FF40
:0F8FFA00F07B017A067979E4F52D7D04028BF97D
:109009009006797422F0A3EFF0A3741CF0A374FF07
:0F901900F07B017A067979E4F52D7D04028BF95D
:10906400E4900679F0A3EFF0A3740AF0A3EFF07B89
:0D907400017A067979E4F52D7D04028BF96F
:0692CB00C2C253E6FD22C1
:1070B300AB37AA38A939853D45853E46853C47AD62
:0570C30036AC35AF34CE
:0C70C8008F3F8C408D418B428A438944ED
:1070D4009006807403F0A374E8F0AD84E4F5842092
:1070E400C7FDC2C4D2C2D2C5E490067FF0F57530A4
:1070F400C3FDAFC1EF24F8602324F8601F24F860B7
:107104003024F8603824F8603924F870030271A43C
:1071140024F870030271A924380271AE90067FE04E
:10712400700BE53F25E044A0F5C27403F0C2C580AE
:107134007CE540F5C290067F7405F0807075750398
:10714400806B90067FE0FFB40509E541F5C2740643
:10715400F0805AEF64067035E5477010AB42054481
:10716400E544AA437002054314F98006AB42AA43DE
:10717400A9441246F7F5C2E546154670021545E5E1
:10718400464545702890067F7407F0802090067F5E
:10719400E0B40707D2C47409F08012757505800D38
:1071A4007575048008757506800375750190067FF2
:1071B400E0B40904C2C38033E575B4031D900680AE
:1071C40074FFF5F012477145F0600FD2C4D2C5D2F6
:1071D400C2C2C3E4F57590067FF0E5756008C2C5C8
:1071E400D2C4C2C38005C2C30270F320C7FD8D841C
:0171F4002278
:0C7699008F348C358D368B378A38893958
:1076A500753C03753DE885843EE4F58420C7FDD22D
:1076B500C2C2C4D2C5E4FFF57530C3FDAEC1EE123A
:1076C50049B176EC0076EF0876EF10771118771947
:1076D50020771E28773430773938773E40774A50FF
:1076E500777358000076EC027779C2C5EF700CE528
:1076F5003425E044A0F5C27F03807CEF64017077F8
:10770500E53425E044A1F5C27F04806BE535F5C27B
:107715007F058063757503805EBF0508E536F5C294
:107725007F068053BF0606D2C57F01804A8011754A
:1077350075048043757506803EBF04047F0280375B
:107745007575058032AB370539E539AA38700205FC
:107755003814F9E5C212473DE53B153B7002153A71
:10776500E53B453A7004C2C2800D7F028009D2C450
:107775007F098003757501BF0904C2C3802FE575B4
:10778500B40319E53D153D7002153C14453C600CEC
:10779500D2C4D2C5D2C2C2C3E4F575FFE57560088F
:1077A500C2C5D2C4C2C38005C2C30276BE20C7FD0E
:0377B500853E848A
:0177B80022AE
:0C7CDA008F348C358D368B378A38893911
:107CE6007E00E536543FFF543F6050C374409FFD0D
:107CF600E49EFCC3E53B9DE53A9C5008853A3D85EC
:107D06003B3E80048C3D8D3E1270B3E57560037F6B
:107D16000222E53E2536F536E53D3535F535E53CB9
:107D2600700CE53E2539F539E53D3538F538C3E5BE
:107D36003B953EF53BE53A953DF53A853A3D853B23
:107D46003ED3E53E9400E53D9400405AE53E94401E
:107D5600E53D940050111270B3E57560037F022271
:107D6600E4F53DF53E80DAAB37AA38A9397545000A
:107D76007546401270BFE57560037F022274C02508
:107D86003EF53E74FF353DF53D74402536F536E447
:107D96003535F535E53C70A974402539F539E435B6
:087DA60038F538027D477F002B
:017DAE0022B2
:1091D800753A00753B01127699E57560037F0122A7
:0391E8007F0022E3
:109184008B747B007A007974753A00753B01E4F5C1
:059194003C127CDA2210
:1091EB0085323A85333B127699E57560037F012210
:0391FB007F0022D0
:0D92280085323A85333BE4F53C127CDA22B6
:0892B00033302E38202020008D
:106E3400C10FC1904106C6004106C7004106CA0001
:106E44004106CB014106CC004106CD004106C800F5
:046E5400C10DC10E9D
:1091990030B30930B2037F28227F292230B2037FFE
:0591A9002A227F2B22A9
:108CE10090063DE0FEA3E0FF900679EEF0A3EFF0E1
:108CF100900643E0FDA3E090067BCDF0A3EDF0EFFD
:108D01004E7012D3E094FF90067BE09400400690F1
:058D110006C77401F02B
:018D1600223A
:10409A0075FFDE75FFADE4F5E6F5E7128A2F20A677
:1040AA00047F0180027F009006C6EFF01289E412B5
:1040BA00894A1291999006C9EFF0C2A790069AE030
:1040CA0025E025E024DAF582E43405F583A3E0FA55
:1040DA00A3E0FFEA4480FAA9079005D2E4F0A3EA34
:1040EA00F0A3E9F0900699E025E025E024FAF582AC
:1040FA00E43405F583A3E0FAA3E0FFEA4480FAA9D1
:10410A00079005D5E4F0A3EAF0A3E9F0E4FF1292E0
:10411A00569006B1E0FF900693E0FD1285AC90063A
:10412A0094E0FF128FCA900695E0FF128EA29006C5
:10413A0096E0FF128E4F900695E0FF128EA290062F
:0C414A0097E0FF128DEA129277127BFBC7
:10415600C207E4F526C20F301E08200705128CE1BF
:10416600D2079006C8E0600BA3E0FF128FEAE49046
:1041760006C8F0201B03024305C21B1284A77F0159
:0F41860012909EEF60419006CBE0602AE4F52591
:1041950074FFF527F528E5281528AE2770021527A1
:0841A500D39400EE940050EEEB
:1041AD000525E525B480E11277B9E49006CBF090B2
:1041BD000695E02402FF128EA27F01128DB6D20E5B
:1041CD007F04128AFEEF601B900696E004F0C39404
:1041DD00034002E4F0900696E0FF90059DF0128EEC
:1041ED004FD20F7F05128AFEEF601B900697E004F9
:1041FD00F0C394034002E4F0900697E0FF90059E13
:10420D00F0128DEAD20F7F07128AFEEF601B900627
:10421D0095E004F0C394084002E4F0900695E0FFA9
:10422D0090059CF0128EA2D20F1291FE8F24900653
:10423D00B1E06524600DE524F0900693E0FD128554
:10424D00ACD20F1291999006C9EFF0E4FF12909E37
:10425D00EF60279006CDE06021E4FF128DB6900649
:10426D00CAE070149006C9E0FF7BFF7A9279B01214
:10427D0088439006CA7401F0D20DE4FF128AFEEF56
:10428D0060419006CDE0601FE49006CAF0300D0449
:10429D00C20D802C900693E06401F0FD9006B1E014
:1042AD00FF1285AC024156E4900693F09006B1E002
:1042BD00FFE4FD1285ACE4FF12924BE49006CCF0C6
:1042CD00127BFB12838AEF6002D20F7F01128AFEEE
:1042DD00EF6022300E04C20E801B900694E004F0B5
:1042ED00C394044002E4F0900694E0FF90059BF027
:1042FD00128FCAD20F128D4D7D157F0112684B7D25
:10430D000E7F0A12684B7D067F0812684B7D037F76
:10431D000912684B7D17E4FF12684B7D167F021260
:10432D00684B7D147F0312684BE4FD7F0412684BCC
:10433D007D017F0512684B7D057F0612684B7D025E
:10434D007F0712684B7D0D7F0B12684B7B017A0640
:10435D00795D128EF2EF70030245EA90065FE0126E
:10436D0049B143F30444400543B114438E16439DB4
:10437D001743BA1A43DC1B43E71D43ED1E000044EF
:10438D00939006937401F09006B1E0FF7D01800CCF
:10439D00E4900693F09006B1E0FFE4FD1285ACD2F7
:1043AD000F0244939006CD7401F00244937B017A81
:1043BD0006795D90066DEBF0A3EAF0A3E9F01246E5
:1043CD00F7FE9006C9E0FF6E6003024493800590EE
:1043DD0006C9E0FF1290090244931292B802449369
:1043ED001292D10244937B017A06795D900670EBAF
:1043FD00F0A3EAF0A3E9F0900003124710FF900636
:10440D00C9E06F6003024493900693E060709006DC
:10441D0070EBF0A3EAF0A3E9F0900005124710FF4E
:10442D00900006124710FD900004124710FB1284F5
:10443D0021804B7B017A06795D900670EBF0A3EA43
:10444D00F0A3E9F0900003124710FF9006C9E06F4A
:10445D007034900693E06026900670EBF0A3EAF0BE
:10446D00A3E9F0900005124710FF900006124710C7
:10447D00FD900004124710FB12823C752601900638
:10448D00C9E0FF129064900693E07003024592908C
:10449D00065FE014603C24FA605B14700302454A29
:1044AD0024F9700302457E240D60030245921250DB
:1044BD001B7B017A06795D90066DEBF0A3EAF0A304
:1044CD00E9F0900003124710FF12924B127BFB0292
:1044DD00457912501B7B017A06795D90066DEBF0E4
:1044ED00A3EAF0A3E9F0900003124710900580F0C5
:1044FD00752601807712501B7B017A06795D900637
:10450D0073EBF0A3EAF0A3E9F0900003124710FF5C
:10451D00900004124710FD900005124710FBC003D8
:10452D00900673E0FBA3E0FAA3E0F99000061247B2
:10453D0010F52CD003128014752601802F12501BFC
:10454D007B017A06795D900673EBF0A3EAF0A3E99F
:10455D00F0900003124710FF900004124710FD90D9
:10456D000005124710FB1264F87526011292358072
:10457D00147B017A06795D900676EBF0A3EAF0A341
:10458D00E9F0127AF8E526640160030243599005BB
:10459D0080E0FF1292569006B1E0FF900693E0FD89
:1045AD001285AC900694E0FF128FCA900695E0FF3D
:1045BD00128EA2900696E0FF128E4F900695E0FFA8
:1045CD00128EA2900697E0FF128DEA129277D2100A
:1045DD0090069BE4F0A304F0C21E024359300F066F
:1045ED00127BFB128D17201003024156127BFBC26A
:0145FD0010AD
:0345FE0002415621
:0A6E58004105B000C116410580009D
:0692D100E49005B0F0225C
:0792B8009005B07401F022E3
:108C6F0090059BE0900694F090059CE0900695F09F
:108C7F0090059DE0900696F090059EE0900697F087
:108C8F0090059FE0900698F09005A0E0900699F06F
:098C9F009005A1E090069AF02274
:108CA800900694E090059BF0900695E090059CF066
:108CB800900696E090059DF0900697E090059EF04E
:108CC800900698E090059FF0900699E09005A0F036
:098CD80090069AE09005A1F0223B
:104FBC00900694E090059BF0900695E090059CF08F
:104FCC00900696E090059DF0900697E090059EF077
:104FDC00900698E090059FF0900699E09005A0F05F
:104FEC0090069AE09005A1F0E4FFEF25E02481F50E
:104FFC0082E43405F583747FF0A374FFF00FBF0DCA
:01500C00E9BA
:01500D002280
:1077B900A2AF9208C2AF90064BE0FCA3E0FDECC477
:1077C900F854F0C868FAEDC4540F48FBECC313FE33
:1077D900ED132BFDEE3AFC90064BE01313543F7E5C
:1077E900002DFFEE3C9005A2F0A3EFF0900649E0D2
:1077F900FCA3E0FDECC4F854F0C868FAEDC4540FDA
:1078090048FBECC313FEED132BFDEE3AFC90064941
:10781900E01313543F7E002DFFEE3C9005A4F0A326
:10782900EFF090062FE0FFA3E09005AACFF0A3EFB9
:10783900F090063BE0FEA3E07802CEC313CE13D846
:10784900F9FF9005AEEEF0A3EFF0900637E0FEA346
:10785900E07802CEC313CE13D8F9FF9005ACEEF051
:10786900A3EFF0900647E0FEA3E0FFC3E49FFF7497
:10787900809EFEEF7803CEA2E713CE13D8F8FF90CF
:1078890005A6EEF0A3EFF0900645E0FEA3E0FFC3E6
:10789900E49FFF74809EFEEF7803CEA2E713CE1318
:1078A900D8F8FF9005A8EEF0A3EFF01292DD7ED094
:1078B9007F007B017A0579A275360075370E128C27
:0878C900341290BAA20892AF3C
:0178D1002294
:10818E00E4F52EF52FF5301292DD7ED07F0F7B00B9
:10819E007A00792F753600753701128C347ED07FB8
:1081AE000E7B007A007930753600753701128C34EB
:1081BE001290BA124FBCE49005A2F0A3F0A3F0A364
:1081CE00F09005AAF0A3F09005AEF0A3F09005ACE8
:1081DE00F0A3F09005A67480F0A3E4F0A37480F0F1
:1081EE00A3E4F01292DD7ED07F007B017A0579A2A6
:1081FE0075360075370E128C341290BA1292DDE479
:10820E00F52D75F021E52DA42400F582E5F034C09E
:10821E00AF82FE7B017A05798175360075372112A2
:0E822E008C34052DE52DC3941E40D70290BA66
:1089E40090D00FE493F4600790D00EE493600512E6
:0489F400818E8031BF
:1089F8007AD07900892C8A2B752AFF752900E52CF5
:108A0800F52CE52BF52BE4F52AF5297B017A057978
:108A1800A2AF2CAE2BAD2AAC29F53475350E128ACF
:018A2800BB92
:068A2900E4900580F0223C
:108D17002016309006CDE06013900693E060249013
:108D270005B0E0701E9006C804F080179006CC745A
:108D370001F0900693F09006B1E0FF7D011285AC3B
:068D4700127BFBD2162294
:108E7900900580E0FFC3941E501EEF75F021A424D5
:108E890000F974C035F0FA7BFF78817C057D017E9D
:098E9900007F211246D1C216220D
:108E1D00900580E0C3941E50281292DD900580E0ED
:108E2D0075F021A42400F582E5F034C0AF82FE7BFD
:108E3D00017A057981753600753721128C341290BF
:028E4D00BA2247
:0692D700128E1DC21622DA
:0B924B00128CA8900580EFF00292D773
:0B925600900580EFF0128E79028C6F03
:048014008D2A8B2BFB
:10801800052C90067BEFF0A3E52BF090067BE0FFA4
:10802800D3952A40030280BF75F021EFA42400F500
:1080380082E5F034C0AF8290067DF0A3EFF09006A1
:108048007CE075F021A42400F582E5F034C0AF820D
:1080580090067FF0A3EFF0E4900679F0A3F0900685
:108068007FE475F001124787AFF0FE90067DE0FCD3
:10807800A3E0F5828C83E493FD12852D90067EE0C3
:1080880004F0700690067DE004F090067AE004F0B3
:108098007006900679E004F0C390067AE094219087
:1080A8000679E0940040B71290BA90067BE004F09D
:1080B800A3E004F0028023900580E0FFE52BD39F26
:0B80C8005009E52CC39F4003129256A4
:0180D300228A
:0664F8008F298D2A8B2B79
:1064FE0090067DE529F0A3E52BF090067DE0D3957F
:10650E002A4003026668A3E075F021A42400F582F8
:10651E00E5F034C0AF82900679F0A3EFF0E4900678
:10652E007FF0A3F090067FE0FEA3E0FFC39421EE80
:10653E0094005038900679E0FCA3E0F5828C83E459
:10654E0093FD74B12FF582E43405F583EDF09006DA
:10655E007AE004F07006900679E004F0900680E090
:10656E0004F070C090067FE004F080B890067DE0E5
:10657E0075F021A42400F582E5F034C0AF829006B8
:10658E007BF0A3EFF090067EE075F021A42400F5D9
:10659E0082E5F034C0AF82900679F0A3EFF0E4907C
:1065AE00067FF0A3F0900679E475F001124787AFED
:1065BE00F0FE90067BE0FCA3E0F5828C83E493FD75
:1065CE0012852D90067CE004F0700690067BE004A8
:1065DE00F0900680E004F0700690067FE004F0C3B1
:1065EE00900680E0942190067FE0940040B79006DC
:1065FE007DE075F021A42400F582E5F034C0AF8271
:10660E0090067BF0A3EFF0E490067FF0A3F09006E7
:10661E007FE0FCA3E0FDC39421EC9400502C900687
:10662E007BE475F001124787AFF0FE74B12DF58251
:10663E00E43405F583E0FD12852D900680E004F02C
:10664E0070CC90067FE004F080C41290BA90067D64
:10665E00E004F0A3E004F0026508900580E0FFE599
:10666E002BD39F501FE529FDE52AC39DFDE4940021
:10667E00FCE52B7A002DFDEA3CFCC3ED9F7480F8FF
:10668E006C985011900580E0FFE529D39F500EE5E0
:0D669E002AC39F4008900580E0FF1292562D
:0166AB0022CC
:06823C008F298D2A8B2B17
:10824200A2AFE433900679F0C2AF1292CBE52AFFD7
:10825200E52990067ECFF0A3EFF0E490067AF09045
:10826200067EE0FCA3E0FD7B017A0579B175320060
:10827200753321AF2B1291EB90067FE02421F09011
:10828200067EE03400F090067AE075F021A4240026
:10829200F974C035F0FAA374FFF0A3EAF0A3E9F091
:1082A2001292DD90067BA3E0FAA3E0AE02FF7B010F
:1082B2007A0579B1753600753721128C341290BA6D
:1082C20090067AE004F0E0C3941E4093900580E0AB
:1082D200FF1292569006C9E0FF12921B900679E0B7
:0482E20024FF92AF34
:0182E6002275
:068421008F298D2A8B2B30
:10842700A2AFE433900679F0C2AF1292CBE52AFFF0
:10843700E52990067BCFF0A3EFF0E490067AF09061
:10844700067AE0FFC3941E504675F021EFA424007E
:10845700F582E5F034C0AF82FE90067DF0A3EFF021
:1084670090067BE0FCA3E0FDAA06A9077BFF753217
:1084770000753321AF2B12922890067CE02421F05F
:1084870090067BE03400F090067AE004F080B0902C
:0F84970006C9E0FF12921B900679E024FF92AF16
:0184A60022B3
:0E920D000001000200040008001000200040D4
:106E620002650032410693004106940041069500F6
:106E72004106960041069700410698004106990096
:106E820041069A0041069D0041069E0041069F0070
:106E92004406A0000000004406A4000000004406CE
:106EA200A8000000004406AC00000000017300428C
:086EB200069B00014106B0003F
:106F6E00900582E02400F556900581E03480F555B9
:106F7E0090058BE0FEA3E07802CEC313CE13D8F9B2
:106F8E00F5548E5390069AE0C39405500E900693D6
:106F9E00E06020E5666432456560189005A6E0FE67
:106FAE00A3E0FFC3E49FF552E49EF551E4F553F5DB
:106FBE00548018900647E06480FEA3E0FF9005A77A
:106FCE00E02FF5529005A6E03EF551900693E06055
:106FDE000AE566643245656002804BC2A790064B97
:106FEE00E0C4F854F0C868FCA3E0C4540F48FD9008
:106FFE00064BE0C313FEA3E0132DFDEE3CFC900602
:10700E004BE01313543F7E002DFDEE3CFC30E704A5
:10701E007C7F7DFF9005A2E0FEA3E0FFC3ED9FFD08
:10702E00EC9EFC30E703E4FCFD75C30E8551C28572
:10703E0052C1E553C313FEE554138E92F591855557
:10704E00C28556C18C928D9175C27F75C1FF8567C1
:10705E0092856891C281C281C281ACCFADCE9006BD
:10706E0095E030E03075C30E75C27F75C1FF8C920E
:10707E008D918563C28564C1E55DC4F854F0C8681E
:10708E00FEE55EC4540F488E92F591C281C281C254
:10709E0081ACCFADCEC3EC648094805003E4FCFD94
:0470AE008C6F8D70E6
:0170B20022BB
:10744F00AB70AA6F75C3038AC28BC1759200759119
:10745F0008C281C281859651859552E552640745D0
:10746F00517068F554755340EA540FFCEB54F075A6
:10747F00C3038CC2F5C1759208759100C281C28198
:10748F00AC96AD95743C2DF58274603CF583E49316
:10749F007A0075C3018AC2F5C1759200759140C219
:1074AF0081C281AA94AB93EB4254EA42537A377B61
:1074BF000075C3018553C28554C18A928B91C281D5
:1074CF00C281AA96AB958A5B8B5C22E4F554E55298
:1074DF0025E0FFE55133FE740D2FF58274923EF5D2
:1074EF0083740193F553EA540FFCEB54F075C30307
:1074FF008CC2F5C1759208759100C281C281AC969C
:10750F00AD95743C2DF58274603CF583E4937A005D
:10751F0075C3018AC2F5C1E55225E0FFE55133FE7F
:10752F00740D2FF58274923EF583E493FE740193EC
:10753F008E92F591C281C281AA94AB93EB4254EA29
:10754F0042537A377B0075C3018553C28554C18A74
:10755F00928B91C281C281AA96AB95EAA2E713FAE8
:06756F00EB138A5BF55CE2
:0175750022F3
:10862A00900597E0F551A3E0F552900637E0FEA3D6
:10863A00E07802CEC313CE13D8F9FF9005ACE0FC64
:10864A00A3E0FDC3EF9DF554EE9CF553900595E02C
:10865A00F555A3E0F55675C30EE42552FFE55134EE
:10866A0080F5C28FC185539285549175C27F75C1B9
:10867A00FFE555C313FEE556138E92F591C281C2EA
:10868A0081C281AFCEAECFC3EE648094805003E442
:06869A00FEFF8E5D8F5E05
:0186A00022B7
:1066AC00900699E0C394055018900645E06480FE6E
:1066BC00A3E0FF9005A9E02FFF9005A8E03EFE8027
:1066CC000F9005A8E0FEA3E0FFC3E49FFFE49EFE4D
:1066DC008E518F52900589E0FEA3E07802CEC31351
:1066EC00CE13D8F9F5548E53900586E02400F55658
:1066FC00900585E03480F555900649E0FCA3E0FD5B
:10670C00ECC4F854F0C868FAEDC4540F48FBECC361
:10671C0013FEED132BFDEE3AFC900649E0131354D7
:10672C003F7E002DFFEE3CFE900691F0A3EFF0EEC5
:10673C0030E70A900691747FF0A374FFF09005A4E3
:10674C00E0FEA3E0FFC3900692E09FFF900691E06D
:10675C009EFEF0A3EFF0EE30E707E4900691F0A375
:0C676C00F0900697E0640260030267F5FD
:10677800856F57857058C3E56A94FFE569943F4073
:1067880027E56A2401FFE56934C0FEEF2558F5586E
:10679800EE3557F557D3E55894FFE557947F401EDB
:1067A80075577F7558FF8016C374FF956AFF743F4D
:1067B8009569FEC3E5589FF558E5579EF55775C38B
:1067C8000E8551C28552C18553928554918555C213
:1067D8008556C1900691E0FEA3E0FF8E928F9175D9
:0B67E800C27F75C1FF85579285589154
:1067F300802D75C30E8551C28552C1855392855430
:10680300918555C28556C1900691E0FEA3E0FF8EA7
:10681300928F9175C27F75C1FF856992856A91C216
:1068230081C281C281900691E5CFF0A3E5CEF090BD
:106833000691E030E707E4900691F0A3F09006910B
:07684300E0F571A3E0F5721E
:01684A00222B
:106B5200AB72AA7175C3038AC28BC175920075911B
:106B620008C281C281859651859552E552640745D6
:106B7200517066F554755340EA540FFCEB54F075AE
:106B8200C3038CC2F5C1759208759100C281C2819E
:106B9200AC96AD95743C2DF58274603CF583E4931C
:106BA2007A0075C3018AC2F5C1759200759140C21F
:106BB20081C281AA94AB93EB4254EA42537A377B67
:106BC2000075C3018553C28554C18A928B91C281DB
:106BD200C281AA96AB95026C73E4F554E55225E0A6
:106BE200FFE55133FE740D2FF58274923EF58374E6
:106BF2000193F553EA540FFCEB54F075C3038CC2B6
:106C0200F5C1759208759100C281C281AC96AD95AD
:106C1200743C2DF58274603CF583E4937A0075C36D
:106C2200018AC2F5C1E55225E0FFE55133FE740D3C
:106C32002FF58274923EF583E493FE7401938E9253
:106C4200F591C281C281AA94AB93EB4254EA4253BA
:106C52007A377B0075C3018553C28554C18A928BF2
:106C620091C281C281AA96AB95EAA2E713FAEB130D
:106C7200FB900697E014603E14603D2402703DAA2A
:036C820071AB7281
:106C850075C3038AC28BC18A928B91C281C28185E9
:106C9500965585955675C3038555C28556C175921A
:106CA50001759100C281C281AA96AB950BBB00010B
:016CB5000AD4
:086CB600800280008A598B5A0C
:016CBE0022B3
:107E820090058FE0F551A3E0F552E42552F55274C6
:107E9200803551F55190063BE0FEA3E07802CEC357
:107EA20013CE13D8F9FF9005AEE0FAA3E0FBC3EFBF
:107EB2009BF554EE9AF553900695E030E12F75C389
:107EC2000E8551C28552C185539285549175C27FE8
:107ED20075C1FFE56BC313FEE56C138E92F59185B8
:107EE20063C28564C1855D92855E91802175C30EF2
:107EF2008551C28552C185539285549175C27F7551
:107F0200C1FFE56BC313FEE56C138E92F591C2813E
:107F1200C281C281ACCFADCEC3EC648094805003E9
:107F2200E4FCFD7466F551F55275C3038CC28DC134
:107F3200855192855291C281C281AC96AD95749958
:097F42002DFD74193CF55F8D6002
:017F4B002213
:0488A100AD07AC066D
:1088A500900633E0FEA3E07806CEC313CE13D8F9C5
:1088B5002401FFEE34FE900691F0A3EFF09006C779
:1088C500E0602D900691E0FEA3E0FFD39400EE64F6
:1088D500809480400FEF2DFDEE3CFC30E7127C7F4D
:1088E5007DFF800CEF2DFDEE3CFC30E703E4FCFD45
:0488F500AE04AF0519
:0188F900225C
:1082E70090058DE0F551A3E0F552900639E0C313F0
:1082F700FEA3E013FF9005AAE0FAA3E0FBC3EF9B00
:10830700F554EE9AF553900695E030E23575C30EB5
:10831700E42552FFE5513480F5C28FC1855392851C
:10832700549175C27F75C1FFE56DC313FEE56E13EA
:108337008E92F5918563C28564C1855D92855E9154
:10834700802775C30EE42552FFE5513480F5C28FAF
:10835700C185539285549175C27F75C1FFE56DC381
:1083670013FEE56E138E92F591C281C281C281AC74
:10837700CFADCEC3EC648094805003E4FCFD8C61E8
:028387008D6205
:0183890022D1
:1071F500201E17C390069BE09420500EA3E004F0D8
:10720500700A90069BE004F08002D21E9006B0E062
:10721500FF04F0EF540364036003027327E573145E
:1072250070030272BA1470030272DE240260030254
:1072350072F0900693E0605AE56664324565603405
:10724500900583E0C313FEA3E013FF9006BDE02F76
:10725500FD9006BCE03EFCE56624CEFFE56534FF07
:10726500FEEF7802C333CE33CED8F92DF568EC3E68
:10727500F5678035900583E0C313FEA3E013FF9007
:1072850006BDE02FF5689006BCE03EF567AF68FEE9
:107295008010900583E0C313F567A3E013F568FF3D
:1072A500AE671288A18E678F68E56730E73DE4F524
:1072B50067F5688036900587E0C313F569A3E01389
:1072C500F56A900591E0F56DA3E0F56EA3E0C313B3
:1072D500F56BA3E013F56C8012D2A7AF84E4F584B7
:1072E500D2EC90065BA3E0F59B8F84E57330E10B50
:1072F50030E008127E82126F6E801DE57330E10862
:107305001266AC12744F8010E57330E005126B52B3
:10731500800612862A1282E70573E573B40403E436
:02732500F573FE
:017327002243
:106EBA0043065501063543065801064541061B009F
:106ECA0041061C0041061D0041061E0042061F0025
:0A6EDA00024206230000C117C11890
:1091AE00AF84E4F58475E881F5BBF5BA75BCA843C8
:0491BE00E7028F84B1
:0191C200228A
:10912400AF8475840275E888E4F5BAF5BB75BCC0F4
:0891340043BC0143E7108F84E6
:01913C002210
:0350300002757690
:10757600C0E0C083C082C0D075D000C000C004C0C7
:0575860005C006C0076E
:10758B00C2ED90061CE0FF25E02425F582E43406CD
:10759B00F583E0FCA3E0FDC3E5BE9D90068EF0E510
:1075AB00BF9C90068DF0E0FCA3E0FDD39400EC644F
:1075BB00809480404A90061BE0FEA807088002C317
:1075CB0013D8FC30E00690061CE0805AD3ED948073
:1075DB00EC64809482500302767A90061CE0FF25BF
:1075EB00E02425F582E43406F583E5BFF0A3E5BE80
:1075FB00F07401A807088002C333D8FC4E806C904E
:10760B00068DE0FEA3E0FFC3EE6480948050609093
:10761B00061CE0FD90061BE0FCA805088002C313C6
:10762B00D8FC20E015ED25E02425F582E43406F5A1
:10763B0083E5BFF0A3E5BEF08035C3EF9480EE6425
:10764B0080947D502A90061CE0FF25E02425F582CE
:10765B00E43406F583E5BFF0A3E5BEF07401A8079B
:10766B00088002C333D8FCFFC3EC9F90061BF0903D
:0B767B00061CE004F05407F0E0F5BB33
:10768600D007D006D005D004D000D0D0D082D08389
:03769600D0E0320F
:035039000269DB2E
:1069DB00C0E0C0F0C083C082C0D075D000C000C082
:0D69EB0001C002C003C004C005C006C00703
:1069F800C2EDAFBE8F488F49900655E0FBA3E0FA81
:106A0800A3E0F990061EE0FF75F002A4F58285F078
:106A18008312479DFDACF0C3E5499D900690F0E5D3
:106A2800489C90068FF0D3A3E0940090068FE06412
:106A3800809480406990061DE0FEA807088002C384
:106A480013D8FC30E014900655E0FBA3E0FAA3E06D
:106A5800F990061EE075F0028074D3900690E094D9
:106A68008090068FE0648094825003026B2B90061E
:106A780055E0FBA3E0FAA3E0F990061EE0FF75F0ED
:106A880002A4F58285F083E5488549F01247F4743D
:106A980001A807088002C333D8FC4E026B27C390B5
:106AA800068FE064809480507A90061EE0FF90067E
:106AB8001DE0FEA807088002C313D8FC20E01F9041
:106AC8000655E0FBA3E0FAA3E0F975F002EFA4F5A0
:106AD8008285F083E5488549F01247F48045C390E4
:106AE8000690E0948090068FE06480947D50349006
:106AF8000655E0FBA3E0FAA3E0F990061EE0FF7557
:106B0800F002A4F58285F083E5488549F01247F440
:106B18007401A807088002C333D8FCFFC3EE9F9016
:0F6B2800061DF090061EE004F05407F0E0F5BBE8
:106B3700D007D006D005D004D003D002D001D000B2
:0B6B4700D0D0D082D083D0F0D0E0325C
:03501500024A0349
:104A0300C0E0C0F0C083C082C0D075D000C000C079
:0D4A130001C002C003C004C005C006C007FA
:104A2000C2FF90061FE0FEA3E0FF20E003024D93CB
:104A3000AD9BA3E0F0A3E04DF0EF64034E7021E0E6
:104A4000C4F8540FC868FF900621E0C454F048F938
:104A5000900658E0FBA3E0FAA3E0C98FF01247D517
:104A600090061FE0FEA3E0FF640F4E6003024B8F31
:104A7000EF24FFFFEE34FFC313FEEF1324FEFFEE1F
:104A800034FFFEEF25E0FFEE33FE900658E0FBA377
:104A9000E0FAA3E0F98F828E8312479DFFE5F0C410
:104AA000F854F0C868FEEFC4540F48FF900621E0A8
:104AB000FCA3E0FDC39FFFEC9EFEA3F0A3EFF0D3A9
:104AC0009400EE64809480405C301703024BFBD36B
:104AD000900624E09403900623E0648094805003C1
:104AE000024D45900622E0C4F8540FC868FD9006B8
:104AF00021E0C454F048FC900620E024FFFF90061B
:104B00001FE034FFC313FEEF1324FEFFEE34FFFE5D
:104B1000EF25E0FFEE338F82F583EC8DF01247F442
:104B2000D217024D45C3900623E064809480400371
:104B3000024D45201703024C6DC3900624E094FDFE
:104B4000900623E06480947F4003024D4590062246
:104B5000E0C4F8540FC868FD900621E0C454F04842
:104B6000FC900620E024FFFF90061FE034FFC313F3
:104B7000FEEF1324FEFFEE34FFFEEF25E0FFEE33E1
:104B80008F82F583EC8DF01247F4C217024D4590E9
:104B9000061FE0FEA3E0FF640D4E6003024CFCEF35
:104BA00024FFFFEE34FFC313FEEF1324FEFFEE34A9
:104BB000FFFEEF25E0FFEE33FE900658E0FBA3E09A
:104BC000FAA3E0F98F828E8312479DFFE5F0C4F8C7
:104BD00054F0C868FEEFC4540F48FF900621E0FC73
:104BE000A3E0FDC39FFFEC9EFEA3F0A3EFF0D394E0
:104BF00000EE64809480406430180BEDC4F8540FCC
:104C0000C868FDEC8076D3900624E09403900623D8
:104C1000E0648094805003024D45900622E0C4F881
:104C2000540FC868FD900621E0C454F048FC90067B
:104C300020E024FFFF90061FE034FFC313FEEF13B4
:104C400024FEFFEE34FFFEEF25E0FFEE338F82F50A
:104C500083EC8DF01247F4D218024D45C390062321
:104C6000E0648094804003024D4520183A9006226B
:104C7000E0C4F8540FC868FD900621E0C454F04821
:104C8000FC900620E024FFFF90061FE034FFC313D2
:104C9000FEEF1324FEFFEE34FFFEEF25E0FFEE33C0
:104CA0008F82F583024D3FC3900624E094FD900669
:104CB00023E06480947F4003024D45900622E0C4C7
:104CC000F8540FC868FD900621E0C454F048FC90E9
:104CD0000620E024FFFF90061FE034FFC313FEEF21
:104CE0001324FEFFEE34FFFEEF25E0FFEE338F824C
:104CF000F583EC8DF01247F4C2188049900622E04B
:104D0000C4F8540FC868FD900621E0C454F048FC74
:104D1000900620E024FFFF90061FE034FFC313FE3F
:104D2000EF1324FEFFEE34FFFEEF25E0FFEE33FE2F
:104D3000900658E0FBA3E0FAA3E0F98F828E83ECA3
:104D40008DF01247F490061FE475F001124771FED2
:104D5000D3E5F09413EE9400401490061FE4F0A302
:104D60007402F090065BE4F0A37484F0804D90062A
:104D700020E024FEFF90061FE034FFFEEF7802C320
:104D800033CE33CED8F94484FF90065BEEF0A3EF28
:104D9000F08028AF9B900621E4F0A3EFF0E0F8E468
:104DA000F0E8900621F090065BE4F0A3F090062076
:0B4DB000E004F0700690061FE004F025
:104DBB00D007D006D005D004D003D002D001D0004C
:0B4DCB00D0D0D082D083D0F0D0E032F6
:106EE400C11B4106B2004106B3FF4806B4000000CE
:056EF400000000000099
:1084A700900679E5B0F0E4A3F090067AE0FFC39474
:0384B700085072F8
:1084BA007401A807088002C333D8FCF5299006790D
:1084CA00E0552924FF92089006B3E0FB5529602E57
:1084DA009006B2E0FE552924FF920920083C2009A3
:1084EA0039E5294EF0E529F4FFEB5FA3F090067A0F
:0C84FA00E024B4F582E43406F583E4F0DD
:10850600801C3008099006B3E04529F080109006DB
:0E8516007AE024B4F582E43406F583E004F044
:0885240090067AE004F0808467
:01852C00222C
:108AFE007401A807088002C333D8FCFF90067BF0F0
:108B0E009006B2E0FE5F601090067BE0FF9006B329
:108B1E00E05F60047F0180027F0090067CEFF060D2
:108B2E000A90067BE0F45E9006B2F090067CE0FFC1
:018B3E002214
:028DB600AB0709
:108DB8007401A807088002C333D8FC90067BF090A2
:108DC80006B2E0FE90067BE0FDF4FCEE5C9006B295
:108DD800F0A3E04DF074B42BF582E43406F583E497
:018DE800F09A
:018DE9002267
:10909E0074B42FF582E43406F583E0D394084003CC
:0B90AE00D38001C39209A209E433FF44
:0190B9002294
:0E91FE00900679E5B0F0E0540C1313543FFFD7
:01920C00223F
:0A926100AF84E4F58475D4978F8480
:01926B0022E0
:0A926C00AF8475840175D4978F84D8
:0192760022D5
:10871600AB84AAB1A2AF921C8F1A8E198D188C1732
:10872600AE19AF1A7877A60608A60753B10FE51853
:10873600700543B110801BE51930E70543B1308061
:108746001143B120431980AE19AF1A7877A60608EF
:10875600A607E4F584C2AF43B701758F037877E6C1
:10876600FE08E6F5828E83E4F053B7FEF58FA21C71
:0687760092AF8AB18B8472
:01877C0022DA
:1086A100AB84AAB1A2AF921D8F108E0F8D0E8C0DCF
:1086B100AF0CEF3395E0FEEFF44E6050AE0FAF100C
:1086C1007879A60608A60753B10FE50E700543B1E8
:1086D10010801BE50F30E70543B130801143B12015
:1086E100430F80AE0FAF107879A60608A607E4F510
:1086F10084C2AF43B701758F017879E6FE08E6F5CC
:10870100828E83E50CF053B7FEE4F58FA21D92AF84
:048711008AB18B841A
:018715002241
:0E8ABB008B2D8A2E892F8F338E328D318C3089
:108AC900E4F536F537C3E5379535E5369534502461
:108AD90078301249541288FAAB2D052FE52FAA2EAA
:108AE9007002052E14F9EF12473D0537E53770D5A9
:048AF900053680D1ED
:018AFD002256
:1088FA00AB84AAB18F3B8E3A8D398C38AE3AAF3BF6
:10890A00787BA60608A60753B10FE539700543B16F
:10891A0010801BE53A30E70543B130801143B1209E
:10892A00433A80AE3AAF3B787BA60608A607787B27
:0F893A00E6FE08E6F5828E83E493FF8AB18B8414
:01894900220B
:108A2F007D017F041287E31290811291C3127DAFF3
:108A3F0012926112926C1291241291AE75F70490FA
:108A4F0006C9E0FF12921B43F6027FB87E2E1290EA
:108A5F00287F997E57128F867FD77E05128FA8D2D7
:088A6F00AFE4F58475D1032288
:1087E300AE8475840F758C20E4F58475EF0675846B
:1087F3000F758A83F59775840F758904F58475B7AA
:108803003075840F4389018D8D758F018F8EFDFC2B
:108813000DBD00010CE4B505F7ECB401F343890287
:10882300E58920E4120DEDAA0470010C14D3940021
:0F883300EA6480948140E9759702E4F58A8E84A7
:018842002213
:10908100AF8475840F75E10375E34075AD0175A576
:0C9091000175A6BF75A04075A4E78F8490
:01909D0022B0
:1091C300E4F584759A73759D1A43E60175F801C237
:0591D30087759B84225A
:107DAF00AE8475840F9006C6E07003027E45C290C4
:107DBF00752900752A10E52A152AAC297002152994
:087DCF00D39400EC940050EE87
:067DD7007F28C286C28570
:107DDD00752900752A10E52A152AAC297002152976
:087DED00D39400EC940050EE69
:027DF500D28535
:107DF700752900752A10E52A152AAC29700215295C
:087E0700D39400EC940050EE4E
:027E0F00DFC8CA
:107E1100752900752A10E52A152AAC297002152941
:087E2100D39400EC940050EE34
:027E2900D290F5
:107E2B00752900752A10E52A152AAC297002152927
:0A7E3B00D39400EC9400403C80EC6E
:067E45007F28C286C28501
:107E4B00752900752A10E52A152AAC297002152907
:087E5B00D39400EC940050EEFA
:027E6300D285C6
:107E6500752900752A10E52A152AAC2970021529ED
:087E7500D39400EC940050EEE0
:047E7D00DFC88E8448
:017E810022DE
:10902800AD84E4F584F5C875C908C39FFFE49EF5CF
:0D903800CB8FCA74FFF5CDF5CCD2CA8D8464
:019045002208
:108F8600AD84758401E4F5C875C908C39FFFE49EE6
:108F9600F5CB8FCA74FFF5CDF5CC43E701D2CA8D68
:018FA6008446
:018FA70022A7
:108FA800AD84758402E4F5C875C908C39FFFE49EC3
:108FB800F5CB8FCA74FFF5CDF5CC43E704D2CA8D43
:018FC8008424
:018FC9002285
:10503C000000000300060009000C000F0012001510
:10504C000019001C001F002200250028002B002F37
:10505C00003200350038003B003E0041004500485E
:10506C00004B004E005100540057005A005E006186
:10507C0000640067006A006D007000730077007AAE
:10508C00007D0080008300860089008C008F0093D7
:10509C0000960099009C009F00A200A500A800AB00
:1050AC0000AE00B200B500B800BB00BE00C100C429
:1050BC0000C700CA00CD00D000D300D700DA00DD55
:1050CC0000E000E300E600E900EC00EF00F200F580
:1050DC0000F800FB00FE010101040107010A010DAB
:1050EC00011001140117011A011D012001230126D1
:1050FC000129012C012F013201350138013B013E00
:10510C000141014401470149014C014F0152015534
:10511C000158015B015E016101640167016A016D67
:10512C000170017301760179017C017E018101849A
:10513C000187018A018D0190019301960199019BD0
:10514C00019E01A101A401A701AA01AD01AF01B209
:10515C0001B501B801BB01BE01C001C301C601C943
:10516C0001CC01CE01D101D401D701DA01DC01DF80
:10517C0001E201E501E801EA01ED01F001F301F5BD
:10518C0001F801FB01FD0200020302060208020BFA
:10519C00020E0210021302160218021B021E02203B
:1051AC00022302260228022B022E02300233023680
:1051BC000238023B023D0240024302450248024AC9
:1051CC00024D024F025202550257025A025C025F14
:1051DC000261026402660269026B026E0270027363
:1051EC0002750278027A027D027F028102840286B5
:1051FC000289028B028E0290029202950297029A09
:10520C00029C029E02A102A302A502A802AA02AD60
:10521C0002AF02B102B302B602B802BA02BD02BFBB
:10522C0002C102C402C602C802CA02CD02CF02D118
:10523C0002D302D502D802DA02DC02DE02E002E37B
:10524C0002E502E702E902EB02ED02F002F202F4DF
:10525C0002F602F802FA02FC02FE03000302030447
:10526C0003070309030B030D030F031103130315AA
:10527C0003170319031B031D031F0321032203241C
:10528C0003260328032A032C032E03300332033492
:10529C00033603370339033B033D033F034103420A
:1052AC00034403460348034A034B034D034F035186
:1052BC0003530354035603580359035B035D035F05
:1052CC00036003620364036503670369036A036C89
:1052DC00036D036F03710372037403750377037813
:1052EC00037A037C037D037F03800382038303859E
:1052FC00038603880389038B038C038D038F039030
:10530C00039203930395039603970399039A039BC4
:10531C00039D039E039F03A103A203A303A503A65E
:10532C0003A703A803AA03AB03AC03AD03AF03B0FD
:10533C0003B103B203B303B503B603B703B803B9A0
:10534C0003BA03BC03BD03BE03BF03C003C103C246
:10535C0003C303C403C503C603C703C803C903CAF5
:10536C0003CB03CC03CD03CE03CF03D003D103D2A5
:10537C0003D303D403D503D603D703D703D803D958
:10538C0003DA03DB03DC03DC03DD03DE03DF03E012
:10539C0003E003E103E203E303E303E403E503E5D2
:1053AC0003E603E703E703E803E903E903EA03EB96
:1053BC0003EB03EC03ED03ED03EE03EE03EF03EF5E
:1053CC0003F003F003F103F103F203F203F303F32D
:1053DC0003F403F403F503F503F603F603F703F7FD
:1053EC0003F703F803F803F803F903F903F903FAD5
:1053FC0003FA03FA03FB03FB03FB03FB03FC03FCB1
:10540C0003FC03FC03FD03FD03FD03FD03FD03FE91
:10541C0003FE03FE03FE03FE03FE03FE03FF03FF76
:10542C0003FF03FF03FF03FF03FF03FF03FF03FF60
:10543C0003FF03FF03FF03FF03FF03FF03FF03FF50
:10544C0003FF03FF03FF03FE03FE03FE03FE03FE45
:10545C0003FE03FE03FD03FD03FD03FD03FD03FC3F
:10546C0003FC03FC03FC03FB03FB03FB03FB03FA3E
:10547C0003FA03FA03F903F903F903F803F803F841
:10548C0003F703F703F703F603F603F503F503F449
:10549C0003F403F303F303F203F203F103F103F058
:1054AC0003F003EF03EF03EE03EE03ED03ED03EC68
:1054BC0003EB03EB03EA03E903E903E803E703E780
:1054CC0003E603E503E503E403E303E303E203E19B
:1054DC0003E003E003DF03DE03DD03DC03DC03DBBB
:1054EC0003DA03D903D803D703D703D603D503D4E0
:1054FC0003D303D203D103D003CF03CE03CD03CC0C
:10550C0003CB03CA03C903C803C703C603C503C43B
:10551C0003C303C203C103C003BF03BE03BD03BC6B
:10552C0003BA03B903B803B703B603B503B303B2A5
:10553C0003B103B003AF03AD03AC03AB03AA03A8E1
:10554C0003A703A603A503A303A203A1039F039E22
:10555C00039D039B039A0399039703960395039367
:10556C0003920390038F038D038C038B03890388B1
:10557C0003860385038303820380037F037D037CFF
:10558C00037A037803770375037403720371036F53
:10559C00036D036C036A03690367036503640362A9
:1055AC000360035F035D035B035903580356035405
:1055BC0003530351034F034D034B034A0348034664
:1055CC00034403420341033F033D033B03390337C9
:1055DC000336033403320330032E032C032A03282F
:1055EC000326032403220321031F031D031B03199A
:1055FC000317031503130311030F030D030B030907
:10560C00030703040302030002FE02FC02FA02F881
:10561C0002F602F402F202F002ED02EB02E902E7FA
:10562C0002E502E302E002DE02DC02DA02D802D575
:10563C0002D302D102CF02CD02CA02C802C602C4F2
:10564C0002C102BF02BD02BA02B802B602B302B175
:10565C0002AF02AD02AA02A802A502A302A1029EF9
:10566C00029C029A0297029502920290028E028B81
:10567C000289028602840281027F027D027A02780C
:10568C00027502730270026E026B0269026602649A
:10569C000261025F025C025A025702550252024F2B
:1056AC00024D024A0248024502430240023D023BBF
:1056BC000238023602330230022E022B0228022656
:1056CC0002230220021E021B0218021602130210F1
:1056DC00020E020B020802060203020001FD01FB8E
:1056EC0001F801F501F301F001ED01EA01E801E532
:1056FC0001E201DF01DC01DA01D701D401D101CED5
:10570C0001CC01C901C601C301C001BE01BB01B876
:10571C0001B501B201AF01AD01AA01A701A401A11C
:10572C00019E019B0199019601930190018D018AC3
:10573C00018701840181017E017C0179017601736D
:10574C000170016D016A016701640161015E015B19
:10575C00015801550152014F014C014901470144C7
:10576C000141013E013B013801350132012F012C71
:10577C000129012601230120011D011A0117011421
:10578C000110010D010A01070104010100FE00FBDB
:10579C0000F800F500F200EF00EC00E900E600E391
:1057AC0000E000DD00DA00D700D300D000CD00CA45
:1057BC0000C700C400C100BE00BB00B800B500B2F9
:1057CC0000AE00AB00A800A500A2009F009C0099B1
:1057DC0000960093008F008C008900860083008067
:1057EC00007D007A007700730070006D006A00671E
:1057FC0000640061005E005A005700540051004ED6
:10580C00004B004800450041003E003B003800358D
:10581C000032002F002B002800250022001F001C46
:10582C00001900150012000F000C000900060003FF
:10583C000000FFFCFFF9FFF6FFF3FFF0FFEDFFEABE
:10584C00FFE6FFE3FFE0FFDDFFDAFFD7FFD4FFD079
:10585C00FFCDFFCAFFC7FFC4FFC1FFBEFFBAFFB732
:10586C00FFB4FFB1FFAEFFABFFA8FFA5FFA1FF9EEA
:10587C00FF9BFF98FF95FF92FF8FFF8CFF88FF85A2
:10588C00FF82FF7FFF7CFF79FF76FF73FF70FF6C59
:10589C00FF69FF66FF63FF60FF5DFF5AFF57FF5410
:1058AC00FF51FF4DFF4AFF47FF44FF41FF3EFF3BC7
:1058BC00FF38FF35FF32FF2FFF2CFF28FF25FF227B
:1058CC00FF1FFF1CFF19FF16FF13FF10FF0DFF0A30
:1058DC00FF07FF04FF01FEFEFEFBFEF8FEF5FEF2E5
:1058EC00FEEFFEEBFEE8FEE5FEE2FEDFFEDCFED99F
:1058FC00FED6FED3FED0FECDFECAFEC7FEC4FEC150
:10590C00FEBEFEBBFEB8FEB6FEB3FEB0FEADFEAAFA
:10591C00FEA7FEA4FEA1FE9EFE9BFE98FE95FE92A7
:10592C00FE8FFE8CFE89FE86FE83FE81FE7EFE7B54
:10593C00FE78FE75FE72FE6FFE6CFE69FE66FE64FE
:10594C00FE61FE5EFE5BFE58FE55FE52FE50FE4DA5
:10595C00FE4AFE47FE44FE41FE3FFE3CFE39FE364B
:10596C00FE33FE31FE2EFE2BFE28FE25FE23FE20EE
:10597C00FE1DFE1AFE17FE15FE12FE0FFE0CFE0A91
:10598C00FE07FE04FE02FDFFFDFCFDF9FDF7FDF434
:10599C00FDF1FDEFFDECFDE9FDE7FDE4FDE1FDDFD3
:1059AC00FDDCFDD9FDD7FDD4FDD1FDCFFDCCFDC96E
:1059BC00FDC7FDC4FDC2FDBFFDBCFDBAFDB7FDB505
:1059CC00FDB2FDB0FDADFDAAFDA8FDA5FDA3FDA09A
:1059DC00FD9EFD9BFD99FD96FD94FD91FD8FFD8C2B
:1059EC00FD8AFD87FD85FD82FD80FD7EFD7BFD79B9
:1059FC00FD76FD74FD71FD6FFD6DFD6AFD68FD6545
:105A0C00FD63FD61FD5EFD5CFD5AFD57FD55FD52CC
:105A1C00FD50FD4EFD4CFD49FD47FD45FD42FD4051
:105A2C00FD3EFD3BFD39FD37FD35FD32FD30FD2ED4
:105A3C00FD2CFD2AFD27FD25FD23FD21FD1FFD1C51
:105A4C00FD1AFD18FD16FD14FD12FD0FFD0DFD0BCD
:105A5C00FD09FD07FD05FD03FD01FCFFFCFDFCFB45
:105A6C00FCF8FCF6FCF4FCF2FCF0FCEEFCECFCEAC2
:105A7C00FCE8FCE6FCE4FCE2FCE0FCDEFCDDFCDB30
:105A8C00FCD9FCD7FCD5FCD3FCD1FCCFFCCDFCCB9A
:105A9C00FCC9FCC8FCC6FCC4FCC2FCC0FCBEFCBD02
:105AAC00FCBBFCB9FCB7FCB5FCB4FCB2FCB0FCAE66
:105ABC00FCACFCABFCA9FCA7FCA6FCA4FCA2FCA0C7
:105ACC00FC9FFC9DFC9BFC9AFC98FC96FC95FC9323
:105ADC00FC92FC90FC8EFC8DFC8BFC8AFC88FC8779
:105AEC00FC85FC83FC82FC80FC7FFC7DFC7CFC7ACE
:105AFC00FC79FC77FC76FC74FC73FC72FC70FC6F1C
:105B0C00FC6DFC6CFC6AFC69FC68FC66FC65FC6466
:105B1C00FC62FC61FC60FC5EFC5DFC5CFC5AFC59AC
:105B2C00FC58FC57FC55FC54FC53FC52FC50FC4FED
:105B3C00FC4EFC4DFC4CFC4AFC49FC48FC47FC462A
:105B4C00FC45FC43FC42FC41FC40FC3FFC3EFC3D64
:105B5C00FC3CFC3BFC3AFC39FC38FC37FC36FC3595
:105B6C00FC34FC33FC32FC31FC30FC2FFC2EFC2DC5
:105B7C00FC2CFC2BFC2AFC29FC28FC28FC27FC26F2
:105B8C00FC25FC24FC23FC23FC22FC21FC20FC1F18
:105B9C00FC1FFC1EFC1DFC1CFC1CFC1BFC1AFC1A38
:105BAC00FC19FC18FC18FC17FC16FC16FC15FC1454
:105BBC00FC14FC13FC12FC12FC11FC11FC10FC106C
:105BCC00FC0FFC0FFC0EFC0EFC0DFC0DFC0CFC0C7D
:105BDC00FC0BFC0BFC0AFC0AFC09FC09FC08FC088D
:105BEC00FC08FC07FC07FC07FC06FC06FC06FC0595
:105BFC00FC05FC05FC04FC04FC04FC04FC03FC0399
:105C0C00FC03FC03FC02FC02FC02FC02FC02FC0197
:105C1C00FC01FC01FC01FC01FC01FC01FC00FC0092
:105C2C00FC00FC00FC00FC00FC00FC00FC00FC0088
:105C3C00FC00FC00FC00FC00FC00FC00FC00FC0078
:105C4C00FC00FC00FC00FC01FC01FC01FC01FC0163
:105C5C00FC01FC01FC02FC02FC02FC02FC02FC0349
:105C6C00FC03FC03FC03FC04FC04FC04FC04FC052A
:105C7C00FC05FC05FC06FC06FC06FC07FC07FC0707
:105C8C00FC08FC08FC08FC09FC09FC0AFC0AFC0BDF
:105C9C00FC0BFC0CFC0CFC0DFC0DFC0EFC0EFC0FB0
:105CAC00FC0FFC10FC10FC11FC11FC12FC12FC1380
:105CBC00FC14FC14FC15FC16FC16FC17FC18FC1848
:105CCC00FC19FC1AFC1AFC1BFC1CFC1CFC1DFC1E0D
:105CDC00FC1FFC1FFC20FC21FC22FC23FC23FC24CD
:105CEC00FC25FC26FC27FC28FC28FC29FC2AFC2B88
:105CFC00FC2CFC2DFC2EFC2FFC30FC31FC32FC333C
:105D0C00FC34FC35FC36FC37FC38FC39FC3AFC3BEB
:105D1C00FC3CFC3DFC3EFC3FFC40FC41FC42FC439B
:105D2C00FC45FC46FC47FC48FC49FC4AFC4CFC4D41
:105D3C00FC4EFC4FFC50FC52FC53FC54FC55FC57E5
:105D4C00FC58FC59FC5AFC5CFC5DFC5EFC60FC6184
:105D5C00FC62FC64FC65FC66FC68FC69FC6AFC6C1F
:105D6C00FC6DFC6FFC70FC72FC73FC74FC76FC77B5
:105D7C00FC79FC7AFC7CFC7DFC7FFC80FC82FC8347
:105D8C00FC85FC87FC88FC8AFC8BFC8DFC8EFC90D3
:105D9C00FC92FC93FC95FC96FC98FC9AFC9BFC9D5D
:105DAC00FC9FFCA0FCA2FCA4FCA6FCA7FCA9FCABE1
:105DBC00FCACFCAEFCB0FCB2FCB4FCB5FCB7FCB962
:105DCC00FCBBFCBDFCBEFCC0FCC2FCC4FCC6FCC8DD
:105DDC00FCC9FCCBFCCDFCCFFCD1FCD3FCD5FCD757
:105DEC00FCD9FCDBFCDDFCDEFCE0FCE2FCE4FCE6CC
:105DFC00FCE8FCEAFCECFCEEFCF0FCF2FCF4FCF63F
:105E0C00FCF8FCFBFCFDFCFFFD01FD03FD05FD07A3
:105E1C00FD09FD0BFD0DFD0FFD12FD14FD16FD180A
:105E2C00FD1AFD1CFD1FFD21FD23FD25FD27FD2A6F
:105E3C00FD2CFD2EFD30FD32FD35FD37FD39FD3BD2
:105E4C00FD3EFD40FD42FD45FD47FD49FD4CFD4E2F
:105E5C00FD50FD52FD55FD57FD5AFD5CFD5EFD618B
:105E6C00FD63FD65FD68FD6AFD6DFD6FFD71FD74E3
:105E7C00FD76FD79FD7BFD7EFD80FD82FD85FD8738
:105E8C00FD8AFD8CFD8FFD91FD94FD96FD99FD9B8A
:105E9C00FD9EFDA0FDA3FDA5FDA8FDAAFDADFDB0D9
:105EAC00FDB2FDB5FDB7FDBAFDBCFDBFFDC2FDC425
:105EBC00FDC7FDC9FDCCFDCFFDD1FDD4FDD7FDD96E
:105ECC00FDDCFDDFFDE1FDE4FDE7FDE9FDECFDEFB3
:105EDC00FDF1FDF4FDF7FDF9FDFCFDFFFE02FE04F6
:105EEC00FE07FE0AFE0CFE0FFE12FE15FE17FE1A32
:105EFC00FE1DFE20FE23FE25FE28FE2BFE2EFE316F
:105F0C00FE33FE36FE39FE3CFE3FFE41FE44FE47AC
:105F1C00FE4AFE4DFE50FE52FE55FE58FE5BFE5EE6
:105F2C00FE61FE64FE66FE69FE6CFE6FFE72FE751F
:105F3C00FE78FE7BFE7EFE81FE83FE86FE89FE8C55
:105F4C00FE8FFE92FE95FE98FE9BFE9EFEA1FEA489
:105F5C00FEA7FEAAFEADFEB0FEB3FEB6FEB8FEBBBB
:105F6C00FEBEFEC1FEC4FEC7FECAFECDFED0FED3F1
:105F7C00FED6FED9FEDCFEDFFEE2FEE5FEE8FEEB21
:105F8C00FEEFFEF2FEF5FEF8FEFBFEFEFF01FF0447
:105F9C00FF07FF0AFF0DFF10FF13FF16FF19FF1C71
:105FAC00FF1FFF22FF25FF28FF2CFF2FFF32FF359D
:105FBC00FF38FF3BFF3EFF41FF44FF47FF4AFF4DC9
:105FCC00FF51FF54FF57FF5AFF5DFF60FF63FF66F1
:105FDC00FF69FF6CFF70FF73FF76FF79FF7CFF7F1B
:105FEC00FF82FF85FF88FF8CFF8FFF92FF95FF9844
:105FFC00FF9BFF9EFFA1FFA5FFA8FFABFFAEFFB16C
:10600C00FFB4FFB7FFBAFFBEFFC1FFC4FFC7FFCA93
:10601C00FFCDFFD0FFD4FFD7FFDAFFDDFFE0FFE3BA
:10602C00FFE6FFEAFFEDFFF0FFF3FFF6FFF9FFFCE1
:10603C000000010202030404050607070809090A07
:10604C000B0C0C0D0E0E0F1011111213141415163F
:10605C00171718191A1A1B1C1D1E1E1F202121226E
:10606C002324252526272829292A2B2C2D2D2E2F94
:10607C003031323233343536373738393A3B3C3DB0
:10608C003D3E3F40414243434445464748494A4BC5
:10609C004B4C4D4E4F5051525354555656575859D0
:1060AC005A5B5C5D5E5F60616263646566676869CC
:1060BC006A6B6C6C6D6E6F707172737475777879C6
:1060CC007A7B7C7D7E7F80818283848586878889AC
:1060DC008A8B8C8E8F9091929394959697989A9B8D
:1060EC009C9D9E9FA0A1A3A4A5A6A7A8A9ABACAD5F
:1060FC00AEAFB0B2B3B4B5B6B7B9BABBBCBDBFC026
:10610C00C1C2C4C5C6C7C8CACBCCCDCFD0D1D2D4DE
:10611C00D5D6D8D9DADBDDDEDFE1E2E3E5E6E7E888
:10612C00EAEBECEEEFF0F2F3F5F6F7F9FAFBFDFE25
:106EF900602005DA000000100080002000D000208A
:106F090000E0002000B0002000C0001000D00020E8
:106F190000E00030602005FA0000001000C00030D9
:106F29000080003000E0003000D0003000C00010C8
:106F390000D0002000E00030C102011100C105C1EC
:106F49000641061A0002120000021400000116048C
:026F5900C180F5
:0350120002503613
:03503600C2CF32B4
:03502D00029046A8
:09904600C0E0C0D075D000C007E5
:0E904F00C2CFAF111511EF7005D21B7511B60F
:07905D00D007D0D0D0E032B3
:0350330002613CDB
:10613C00C0E0C0F0C083C082C0D075D000C000C029
:0D614C0001C002C003C004C005C006C007AA
:1061590085B14AC2CF7584031271F5900694E01493
:10616900606224FE7003026218046003026225D291
:1061790000E51254E0FE7F0070047D0180027D007D
:10618900A20CE4335DFDE4B50708EEB4E0047F0139
:1061990080027F00EF4D6019E51430E703D38001D9
:1061A900C3920BA203B00B5008751200751300C2FD
:1061B9000CA20B9203D3E5139400E51294E0405C22
:1061C900D20C8058E51220E7047F0180027F00A2EB
:1061D9000CE4335FFFE51230E7047E0180027E00A4
:1061E900EE4F6018E51430E703D38001C3920BA288
:1061F90003B00B5007A200B39200C20CA20B92038A
:10620900D3E5139400E51294E04011D20C800DD22D
:1062190000300108751200751300C201900697E05D
:10622900FD7008D51623751604800330000EE55A53
:106239002513F513E5593512F512800DC3E51395AC
:106249005AF513E5129559F512900696E014604136
:106259001460302402704DE51220E711E51325E0A2
:10626900FFE51233FEEF2401F54CEE801EE5132500
:10627900E0FFE51233FEC374FF9FF54C747F9EF572
:106289004B8021E5132401F54CE5123480F54B8050
:1062990013E51220E708754B7F754CFF8006754B97
:1062A90080754C01854B63854C649006C6E060554A
:1062B900E56330E704D2058002C205A20530060174
:1062C900B3503E9006CFE054FCF0ED70053005194F
:1062D9008029900697E0B40226900587E0FCA3E0A8
:1062E900FDD39400EC948140099006CFE04401F07D
:1062F900800DC3EC947F50079006CFE04402F0D2A2
:1063090010A2059206758400634B80854BD3854C9A
:10631900D2758403E55C2515F515E55B3514F5148F
:10632900E515AE147805CEC313CE13D8F9F54C8E06
:106339004B25E0FFE54B33FE743C2FF58274503E4C
:10634900F583E493F54B740193F54C75C303854BC1
:10635900C2854CC1855F92856091C281C281859653
:106369004B85954CE4254CF54C7404354BF54B9015
:10637900069AE0FD7014E54CC4F8540FC868F54E50
:10638900E54BC454F048F54D8072EDC39405502493
:1063990053B10F9005D8E042B19005D2A3E0FAA31A
:1063A900E0F582E54C25E0FFE54B33FEE5822FF56C
:1063B90082EA803953B10F9005D8E042B19006477F
:1063C900E0FEA3E07802CEC313CE13D8F9FF9005FF
:1063D9008CE02FFF90058BE03E8F82F583E54C25FD
:1063E900E0FFE54B33FEE5822FF582E5833EF58339
:1063F900E493F54D740193F54E854AB1900699E001
:10640900FD7014E54CC4F8540FC868F550E54BC449
:1064190054F048F54F8072EDC39405502453B10FE1
:106429009005D9E042B19005D5A3E0FAA3E0F58241
:10643900E54C25E0FFE54B33FEE5822FF582EA8046
:106449003953B10F9005D9E042B1900645E0FEA35A
:10645900E07802CEC313CE13D8F9FF90058AE02F56
:10646900FF900589E03E8F82F583E54C25E0FFE545
:106479004B33FEE5822FF582E5833EF583E493F500
:106489004F740193F550854AB1E56130E7067561AE
:1064990000756200C374FF9562F54C747F9561F5D0
:1064A9004B75C30E8561C28562C1854D92854E913A
:1064B900854BC2854CC1854F92855091C281C2815D
:1064C900C28185CF4B85CE4C634B80758401854B4A
:0464D900D3854CD249
:1064DD00D007D006D005D004D003D002D001D00013
:0B64ED00D0D0D082D083D0F0D0E032BD
:026F5B00C11E55
:084DD6008F2D8E2C8D2B8C2AF1
:104DDE00C3E5319535FFE5309534FEE52F9533FD6E
:104DEE00E52E9532FC90067912497490067D124993
:104DFE008000000000900679E0FCEC334003024E88
:104E0E00BCAF35AE34AD33AC32900689124974E482
:104E1E007F01FEFDFC900689E0F8A3E0F9A3E0FA1D
:104E2E00A3E0FBC312493E500A9006891249800046
:104E3E00000001AF2DAE2CAD2BAC2AAB39AA38A990
:104E4E0037A836124821C004C005C006C007900618
:104E5E0089E0FCA3E0FDA3E0FEA3E0FBAA06A90502
:104E6E00A804D007D006D005D0041248AC90068115
:104E7E00124974900681E0FCA3E0FDA3E0FEA3E0DE
:104E8E00FFAB31AA30A92FA82E1248219006851209
:104E9E004974900685E0FCA3E0FDA3E0FEA3E0FFCD
:104EAE00AB39AA38A937A8361248AC024FABE4FF8B
:104EBE00FEFDFC900679E0F8A3E0F9A3E0FAA3E08A
:104ECE00FBD312493E5003024FB1E539952DFFE554
:104EDE0038952CFEE537952BFDE536952AFCAB393A
:104EEE00AA38A937A836124821900681124974C3F0
:104EFE00E5399535FFE5389534FEE5379533FDE513
:104F0E00369532FC900689124974E47F01FEFDFC51
:104F1E00900689E0F8A3E0F9A3E0FAA3E0FBC31240
:104F2E00493E500A90068912498000000001900601
:104F3E0081E0FCA3E0FDA3E0FEA3E0FF900689E084
:104F4E00F8A3E0F9A3E0FAA3E0FB128A77900681BA
:104F5E00124974C3E5399531FBE5389530FAE537DA
:104F6E00952FF9E536952EF8900681E0FCA3E0FD2D
:104F7E00A3E0FEA3E0FF124821AB39AA38A937A857
:104F8E00361248ACAB07AA06A905A804C3E5399B9F
:104F9E00FFE5389AFEE53799FDE53698FC90067DDB
:0D4FAE0012497490067DA3A3E0FEA3E0FF6E
:014FBB0022D3
:1080D4008C2A8D2BA907E925E0244CF582E434058C
:1080E400F583E0FEA3E0C3952BEE952A5027E925FE
:1080F400E0244CF582E43405F583E52AF0A3E52B6E
:10810400F024E2FFE52A34FFFEE925E02466F58247
:10811400E43405804BE925E02466F582E43405F572
:1081240083E0FEA3E0D3952BEE952A403AE925E0BF
:108134002466F582E43405F583E52AF0A3E52BF003
:10814400E925E02466F582E43405F583E0FEA3E046
:10815400241EFFE43EFEE925E0244CF582E43405C8
:10816400F583EEF0A3EFF0E925E02466F582E4342C
:1081740005F583E0F52AA3E0F52BD39BE52A9A4085
:0A818400048A2A8B2BAE2AAF2B22AF
:02684B008F2993
:10684D00EF25E02432F582E43405F583E0FFA3E083
:10685D00900526CFF0A3EFF0ED25E02425F582E499
:10686D003406F583E0FFA3E0900522CFF0A3EFF00F
:10687D00900522E0C4F854F0C868FCA3E0C4540F9E
:10688D0048FD7BFF7A0FAF291280D4900524EEF0DE
:10689D00A3EFF0E0C4F8540FC868F0900524E0C4ED
:1068AD0054F048F0A3E054F0F0E52925E02481F5FB
:1068BD0082E43405F583E0C4F854F0C868FFA3E022
:1068CD00C4540F4890052ACFF0A3EFF0900524E0B3
:1068DD00FCA3E0FDECC4F854F0C868FFEDC4540F00
:1068ED004890052CCFF0A3EFF0900526E0FAA3E039
:1068FD00FBEAC4F854F0C868FFEBC4540F48900588
:10690D002ECFF0A3EFF0A3740FF0A374FFF0ED6B97
:10691D007002EC6A70030269DA90052AE0FEA3E0CA
:10692D00FFE4FCFDC006C007A3E0FEA3E0FFE48F7B
:10693D00318E30F52FF52EA3E0FEA3E0FFE48F3569
:10694D008E34F533F532A3E0FEA3E0FFE48F398EEC
:10695D0038F537F536D007D006124DD6900528EE0E
:10696D00F0A3EFF0E0C4F8540FC868F0900528E0EC
:10697D00C454F048F0A3E054F0F0E52925E024815B
:10698D00F582E43405F583E0FEA3E0FF900528E0F1
:10699D00FCA3E0FD6F7002EC6E6018E52925E02484
:1069AD0081F582E43405F583ECF0A3EDF0301E03A0
:1069BD00128D17900524E0FEA3E0FFE52925E024C4
:0D69CD0032F582E43405F583EEF0A3EFF01F
:0169DA00229A
:09928C00900583EEF0A3EFF0223F
:09929500900595EEF0A3EFF02224
:09929E00900591EEF0A3EFF0221F
:0992A700900593EEF0A3EFF02214
:04500E000604020092
:0E6F5D004506CF0000000000C11F4106CE0017
:108B7F00E4F52A530707EF540390500E93FEEFC30B
:108B8F00940450159006D3E0FFEDA806088002C3A9
:108B9F0033D8FC4F9006D3F0229006D2E0FFEDA819
:0D8BAF0006088002C333D8FC4F9006D2F0B8
:018BBC002296
:1090F1009006CFE0FE5306F3EF60047F0880027F05
:0991010004EF42069006CFEEF0E7
:01910A002242
:107F4C0090069AE0D3940440047F0180027F008F56
:107F5C0029900699E0D3940440047F0180027F00AD
:107F6C00AC07E49006D2F0A3F090069AE09005A13D
:107F7C00F025E025E024DAF582E43405F583A3E06E
:107F8C00FAA3E0FFEA4480FAA9079005D2E4F0A333
:107F9C00EAF0A3E9F090069AE0FF25E025E024DD65
:107FAC00F582E43405F583E09005D8F07D01128B61
:107FBC007F900699E0FF9005A0F00D128B7F900644
:107FCC0099E0FF25E025E024FAF582E43405F583F9
:107FDC00A3E0FAA3E0FBEA4480FAA9039005D5E4F8
:107FEC00F0A3EAF0A3E9F0EF25E025E024FDF5820B
:107FFC00E43405F583E09005D9F09006C6E06007FF
:07800C00AF04AD291290D66C
:01801300224A
:0B927700900698E0FF1290F1027F4C7F
:10838A00C208E4900679F0A3F07F0612909EEF608F
:10839A00267F06128DB6201F1A900698E070047F79
:1083AA000180027F00900698EFF090059FF01290EE
:1083BA00F1D208D21F80267F06128AFEEF601E3095
:1083CA001F04C21F8017900698E0700590069A80D5
:1083DA0003900699E004F0E05407F0D208127F4CAB
:1083EA009006C6E0602B900699E0C394054006907B
:1083FA00067A7401F090069AE0C394054006900646
:10840A00797401F090067AE0FF900679E0FD129007
:06841A00D6A208E433FFC6
:018420002239
:1085AC00AC079006D1E05430F0ED603A9006C6E08E
:1085BC006002800EEC14601214601714601A24030D
:1085CC00705B9006D1E04402F0229006D1E04408A2
:1085DC00F0229006D1E0800A9006D1E04402F044EB
:1085EC0008F04480F0229006C6E07031EC14601262
:1085FC0014601714601A240370239006D1E0440110
:10860C00F0229006D1E04404F0229006D1E0800ADA
:0E861C009006D1E04401F04404F04440F02206
:1090D600AE079006D1E054CFF0EE6004E04410F005
:0B90E600ED60079006D1E04420F0226E
:108E4F009006CFE0548FF0EF14600F1460142402DB
:108E5F0070179006CFE04440F0229006CFE04420F8
:0A8E6F00F0229006CFE04410F0223C
:108EA200AD079006D0E054E3F0ED30E004E044106A
:108EB200F0ED30E1079006D0E04408F0ED30E20733
:088EC2009006D0E04404F02208
:108DEA00AD079006D0E054FCF09006CFE0547FF037
:108DFA00ED14600F146014240270179006CFE0443B
:108E0A0080F0229006D0E04401F0229006D0E0449F
:038E1A0002F02241
:108ECA00AD079006D0E0541FF0ED30E004E0448096
:108EDA00F0ED30E1079006D0E04440F0ED30E207D3
:088EEA009006D0E04420F022C4
:108FCA00EF14601214601314600824037011E4FF94
:108FDA00800A7F0480067F0180027F02128ECA22E5
:108D4D00900679E561F0A3E562F0900679E0900672
:108D5D007BF0E0FFC374FF9FF0E0C313FFF09006BC
:108D6D00CEE06F600F90067BE0FF9006CEF053A033
:048D7D00C0EF42A061
:018D810022CF
:108F3D00EF540314600F146014240270179006CFC1
:108F4D00E054FCF0229006CFE04402F0229006CFD0
:058F5D00E04401F022D8
:107BFB0090067BE584F075840F9006C6E0601AC290
:017C0B0090E8
:107C0C00752A00752B10E52B152BAE2A7002152A40
:087C1C00D39400EE940050EE39
:107C2400E4900679F0900679E0FFC39405400302DE
:027C34007CB31F
:107C360074CF2FF582E43406F583E0F52AE4900646
:0C7C46007AF090067AE0FFC394085058D2
:107C520074017E00A807088005C333CE33CED8F95D
:0E7C6200FFEF552A24FF9208A2089286C285E1
:107C7000752B00752C10E52C152CAE2B7002152BD6
:087C8000D39400EE940050EED5
:027C8800D285A3
:107C8A00752B00752C10E52C152CAE2B7002152BBC
:087C9A00D39400EE940050EEBB
:087CA20090067AE004F0809ED8
:0F7CAA00900679E004F0027C299006C6E0601A8B
:107CB900752A00752B10E52B152BAE2A7002152A93
:087CC900D39400EE940050EE8C
:087CD100D29090067BE0F584DF
:017CD9002288
:10894A009006C6E06008D290E4FDFF1290D6900629
:10895A00B1E0FF900693E0FD1285AC900694E0FF2B
:10896A00128FCA900695E0FF128EA2900696E0FF3B
:10897A00128E4FE4FF128F3D900695E0FF128EA2F1
:0E898A00900697E0FF128DEA129277027BFBB7
:10915500000002AB055508000AAB0D55100012AB17
:08916500155518001AAB1D5549
:026F6B00C1194A
:0278D200A90704
:1078D400E975F00C84ABF07A00E975F00C8424FFB0
:1078E400F533E434FFF532EA6003027984EBB40C37
:1078F400004003027984907901F8282873027925DD
:1079040002792B02793102793702793D02794302F7
:10791400794902794F02795502795B0279680279D3
:10792400767A007B03805D7A007B0480577A007B43
:107934000580517A007B06804B7A007B0780457A6C
:10794400007B08803F7A007B0980397A007B0A80BB
:10795400337A007B0B802DE4FAFB0533E533702486
:10796400053280207A007B010533E5337016053239
:1079740080127A007B020533E533700805328004F7
:10798400E4FEFF22E533C43354E0FEE4F5318E30E7
:10799400F52FF52EEB25E0FFEA33FE74552FF58223
:1079A40074913EF583E493FE740193FFE4FCFDE5DA
:1079B400312FF531E5303EF530ED352FF52FEC352F
:1079C4002EF52EE9D394674009E47531FF7530FF35
:1079D400800BE9C394095009E4F531F530F52FF52E
:0579E4002EAE30AF31B2
:0179E900227B
:1079EA008D1BEF14604A24ECB40B004003027AF2B8
:1079FA00907A0875F003A4C58325F0C58373027ACB
:107A0A0029027AF2027A4C027A5D027A60027A7D5F
:107A1A00027A9A027AA5027AB8027ACB027ADEE56B
:107A2A001B75F00A84FF900694F0128FCA7F012218
:0F7A3A00E51B25E0F51BF51CAF1DAE1C12929548
:107A49007F0122E51B75F00A84FF900695F0128EDE
:107A5900A27F01227F0022E51B75F00A8490069718
:107A6900F0D3940240037402F0900697E0FF128D60
:107A7900EA7F0122E51B75F00A84900696F0D394FB
:107A89000240037402F0900696E0FF128E4F7F01C8
:107A990022E51B75F00A849006998009E51B75F0AB
:107AA9000A8490069AF05407F0127F4C7F0122E570
:107AB9001B25E0F51B751B00AF1B7E0012929E7FF4
:107AC9000122E51B25E0F51B751B00AF1B7E00128B
:107AD90092A77F0122E51BFD7C0075F004A4AEF09E
:0F7AE9002DF566EC3EF56580037F00227F0022BD
:067AF8008B298A2A892B6C
:107AFE00900003124710900679F0E0FD540FA3F0AA
:107B0E00FC9006B1E0FF74017E00A807088005C353
:107B1E0033CE33CED8F9FFECFBEF5B24FF9208EDAA
:107B2E0054F02450603424D0606424F07003027B3F
:0E7B3E00F824606003027BF8200803027BF845
:107B4C00AB29AA2AA92B900005124710FF1278D254
:097B5C008E2C8F2D12928CD201A7
:107B6500027BF8200803027BF8AB29AA2AA92B90EF
:107B75000005124710641F707A90000612471075B1
:107B85006500F566D39433E56594004066E56615B2
:107B95006670601565805C300859AB29AA2AA92B47
:107BA50090000612471025E09006C4F0A3E4F0907B
:107BB500000512471075F004A4FF9006C4E045F0D7
:107BC500FEA3E04FFF9006C4EEF0A3EFF02401FF03
:107BD500EE34809006BCF0A3EFF09006BCE0FEA367
:107BE500E07803CEA2E713CE13D8F8F0EE9006BCEA
:057BF500F080007F009C
:017BFA002268
:108B3F00AB84A2AF9209E4FDED8F3F8E3EF53DF57C
:108B4F003CAE3EAF3F787BA60608A607F584C2AFC2
:108B5F0043B701438F02438F0118E6FE08E6F58203
:0F8B6F008E83E4F053B7FEF58FA20992AF8B848B
:018B7E0022D4
:02899800AB052D
:10899A00AA84A2AF9209E4FDED8F458E44F543F512
:1089AA0042EBFF3395E0FEEFF44E6027AE44AF454D
:1089BA00787BA60608A607E4F584C2AF43B701751B
:1089CA008F0118E6FE08E6F5828E83EBF053B7FEB8
:0989DA00E4F58FA20992AF8A8432
:0189E3002271
:108BBD008E3C8F3D8C3E8D3F8A408B41E54145403B
:108BCD006029853F82853E83E0FDAF3DAE3C128935
:108BDD0098E541154170021540053FE53F700205CE
:0C8BED003E053DE53D70D5053C80D122E1
:0692DD00E4F51EF51F225E
:1090BA00AF1FAE1E128B3F7C007D007B007A04AF8F
:0C90CA001FAE1E128BBDE4F51EF51F2228
:06852D008E388F39A9050C
:10853300EE54FCFEE51F7003EE651E6059E51F4512
:108543001E60031290BAE53854FCF51E751F00F542
:108553003A851F3B7E007F009006817404F0A3E4FC
:10856300F0053BE53BAC3A7002053A14F5828C8387
:10857300E493FD0FEFAA0670010E14F5828A83EDD2
:10858300F0900682E024FFF0900681E034FFF0E0F3
:108593007002A3E070CBE5385403FE74002539F56F
:0885A3008274003EF583E9F04B
:0185AB0022AD
:108C34008E318F328B338A348935E5371537AE362A
:108C4400700215364E60230532E532AE31700205EE
:108C54003114FFAB330535E535AA347002053414FD
:0B8C6400F91246F7FD12852D80D0228A
:03000000024000BB
:03000300025003A5
:03000B000250069A
:030013000250098F
:03001B0002500C84
:0300230002500F79
:03002B000250126E
:0300330002501563
:03003B0002501858
:0300430002501B4D
:03004B0002501E42
:0300530002502137
:03005B000250242C
:0300630002502721
:03006B0002502A16
:0300730002502D0B
:03007B0002503000
:03008300025033F5
:03008B00025036EA
:03009300025039DF
:03009B0002503CD4
:0300A30002503FC9
:10400000787FE4F6D8FD9000007F007E20E4F0A3E6
:0A401000DFFCDEFA75817C024055EA
:10401A0002409AE493A3F8E493A34003F68001F2E2
:10402A0008DFF48029E493A3F85407240CC8C333A7
:10403A00C4540F4420C8834004F456800146F6DF76
:10404A00E4800B0102040810204080906E1FE47E79
:10405A00019360BCA3FF543F30E509541FFEE4936B
:10406A00A360010ECF54C025E060A840B8E493A332
:10407A00FAE493A3F8E493A3C8C582C8CAC583CA5D
:10408A00F0A3C8C582C8CAC583CADFE9DEE780BE15
:016F6D000023
:10460100E709F608DFFA8046E709F208DFFA803E9B
:1046110088828C83E709F0A3DFFA8032E309F60888
:10462100DFFA8078E309F208DFFA807088828C83F0
:10463100E309F0A3DFFA806489828A83E0A3F608A4
:10464100DFFA805889828A83E0A3F208DFFA804C7E
:1046510080D280FA80C680D4806980F28033801055
:1046610080A680EA809A80A880DA80E280CA8033BE
:1046710089828A83ECFAE493A3C8C582C8CCC58336
:10468100CCF0A3C8C582C8CCC583CCDFE9DEE78006
:104691000D89828A83E493A3F608DFF9ECFAA9F085
:1046A100EDFB2289828A83ECFAE0A3C8C582C8CCDB
:1046B100C583CCF0A3C8C582C8CCC583CCDFEADEF4
:1046C100E880DB89828A83E493A3F208DFF980CC56
:1046D10088F0EF60010E4E60C388F0ED2402B4044F
:1046E1000050B9F582EB2402B4040050AF232345F6
:0646F10082239046517384
:1046F700BB010689828A83E0225002E722BBFE02C1
:09470700E32289828A83E49322F3
:10471000BB010CE58229F582E5833AF583E022505E
:1047200006E92582F8E622BBFE06E92582F8E222A8
:0D473000E58229F582E5833AF583E49322C2
:10473D00BB010689828A83F0225002F722BBFE015B
:02474D00F32255
:10474F00F8BB010DE58229F582E5833AF583E8F0A0
:10475F00225006E92582C8F622BBFE05E92582C84C
:02476F00F22234
:10477100C5F0F8A3E028F0C5F0F8E58215827002D3
:064781001583E038F02270
:10478700A3F8E0C5F025F0F0E582158270021583E5
:06479700E0C838F0E82242
:10479D00BB0110E58229F582E5833AF583E0F5F05A
:1047AD00A3E0225009E92582F886F008E622BBFE37
:1047BD000AE92582F8E2F5F008E222E5832AF5837D
:0847CD00E993F5F0A3E9932242
:1047D500BB010A89828A83F0E5F0A3F0225006F72F
:0F47E50009A7F01922BBFE06F3E5F009F319222C
:1047F400F8BB0111E58229F582E5833AF583E8F0F7
:10480400E5F0A3F0225009E92582C8F608A6F022B3
:0D481400BBFE09E92582C8F2E5F008F2229A
:10482100E88FF0A4CC8BF0A42CFCE98EF0A42CFC36
:104831008AF0EDA42CFCEA8EF0A4CDA8F08BF0A4B4
:104841002DCC3825F0FDE98FF0A42CCD35F0FCEB13
:104851008EF0A4FEA9F0EB8FF0A4CFC5F02ECD39D8
:0F486100FEE43CFCEAA42DCE35F0FDE43CFC2245
:1048700075F008758200EF2FFFEE33FECD33CDCCFF
:1048800033CCC58233C5829BED9AEC99E582984082
:104890000CF582EE9BFEED9AFDEC99FC0FD5F0D65F
:1048A000E4CEFBE4CDFAE4CCF9A88222B800C1B989
:1048B0000059BA002DEC8BF084CFCECDFCE5F0CBC7
:1048C000F97818EF2FFFEE33FEED33FDEC33FCEB00
:1048D00033FB10D703994004EB99FB0FD8E5E4F9BB
:1048E000FA227818EF2FFFEE33FEED33FDEC33FCA8
:1048F000C933C910D7059BE99A4007EC9BFCE99A9C
:10490000F90FD8E0E4C9FAE4CCFB2275F010EF2FE0
:10491000FFEE33FEED33FDCC33CCC833C810D707E0
:104920009BEC9AE899400AED9BFDEC9AFCE899F81B
:0E4930000FD5F0DAE4CDFBE4CCFAE4C8F922AE
:108A7700C2D5E830E70FB2D5E4C39BFBE49AFAE42A
:108A870099F9E498F8EC30E717B2D5128AAD124895
:108A9700ACE4C39BFBE49AFAE499F9E498F8800301
:108AA7001248AC30D50DE4C39FFFE49EFEE49DFD64
:048AB700E49CFC221D
:10493E00EB9FF5F0EA9E42F0E99D42F0EC6480C8F0
:06494E0064809845F02290
:104954007401FF3395E0FEFDFC080808E6CF2FF64E
:1049640018E6CE3EF618E6CD3DF618E6CC3CF62227
:0C497400ECF0A3EDF0A3EEF0A3EFF022B6
:10498000A8828583F0D083D082124997124997126A
:104990004997124997E473E493A3C583C5F0C5838F
:1049A000C8C582C8F0A3C583C5F0C583C8C582C881
:0149B00022E4
:1049B100D083D082F8E4937012740193700DA3A395
:1049C10093F8740193F5828883E4737402936860A9
:0649D100EFA3A3A380DFA9
:1049D700EF4E6012EF60010EEDBB010B89828A83F7
:1049E700F0A3DFFCDEFA2289F05007F709DFFCA904
:0C49F700F022BBFEFCF309DFFCA9F0225B
:00000001FF
